:100000000C9462000C948A000C948A000C948A0070
:100010000C948A000C948A000C948A000C948A0038
:100020000C948A000C948A000C948A000C948A0028
:100030000C948A000C948A000C948A000C948A0018
:100040000C945E030C948A000C94CE030C94A803C9
:100050000C948A000C948A000C948A000C948A00F8
:100060000C948A000C948A000000000024002700F1
:100070002A0000000000250028002B0000000000DE
:1000800023002600290004040404040404040202DA
:100090000202020203030303030301020408102007
:1000A0004080010204081020010204081020000012
:1000B0000008000201000003040700000000000027
:1000C0000000F50511241FBECFEFD8E0DEBFCDBF85
:1000D00011E0A0E0B1E0E8E9FCE002C005900D927B
:1000E000AA31B107D9F721E0AAE1B1E001C01D9220
:1000F000A53FB207E1F710E0C2E6D0E004C02197C7
:10010000FE010E944406C136D107C9F70E940004CF
:100110000C944A060C940000833081F028F481305E
:1001200099F08230A9F008958730A9F08830C9F09D
:100130008430B1F4809180008F7D03C08091800075
:100140008F7780938000089584B58F7784BD08955C
:1001500084B58F7DFBCF8091B0008F778093B00006
:1001600008958091B0008F7DF9CF1F93CF93DF93D7
:10017000282F30E0F901E255FF4F8491F901E6564E
:10018000FF4FD491F901EA57FF4FC491CC23A9F056
:10019000162F81110E948C00EC2FF0E0EE0FFF1F54
:1001A000EE58FF4FA591B4918FB7F894EC911111CF
:1001B00008C0D095DE23DC938FBFDF91CF911F91D4
:1001C0000895DE2BF8CFCF93DF9390E0FC01E65645
:1001D000FF4F24918A579F4FFC0184918823D1F0CF
:1001E00090E0880F991FFC01E859FF4FA591B49149
:1001F000FC01EE58FF4FC591D49161110EC09FB71D
:10020000F8948C91E22FE0958E238C932881E22341
:10021000E8839FBFDF91CF9108958FB7F894EC9159
:10022000E22BEC938FBFF6CFAF92BF92CF92DF92CB
:10023000EF92FF920F931F93CF93DF936C017B019B
:100240008B01040F151FEB015E01AE18BF08C0172C
:10025000D10759F06991D601ED91FC910190F0819F
:10026000E02DC6010995892B79F7C501DF91CF9162
:100270001F910F91FF90EF90DF90CF90BF90AF90C4
:100280000895FC01538D448D252F30E0842F90E09C
:10029000821B930B541710F0CF9608950197089581
:1002A000FC01918D828D981761F0A28DAE0FBF2F4A
:1002B000B11D5D968C91928D9F5F9F73928F90E0A0
:1002C00008958FEF9FEF0895FC01918D828D98170F
:1002D00031F0828DE80FF11D858D90E008958FEF4C
:1002E0009FEF0895FC01918D228D892F90E0805C15
:1002F0009F4F821B91098F739927089588E591E09C
:100300000E94720121E0892B09F420E0822F0895D8
:1003100080E090E0892B29F00E947E0181110C94ED
:1003200000000895FC01A48DA80FB92FB11DA35A98
:10033000BF4F2C91848D90E001968F739927848F05
:10034000A689B7892C93A089B1898C918370806428
:100350008C93938D848D981306C00288F389E02DC9
:1003600080818F7D80830895EF92FF920F931F937A
:10037000CF93DF93EC0181E0888F9B8D8C8D981358
:100380001AC0E889F989808185FF15C09FB7F89464
:10039000EE89FF896083E889F989808183708064B0
:1003A00080839FBF81E090E0DF91CF911F910F91FB
:1003B000FF90EF900895F62E0B8D10E00F5F1F4F0A
:1003C0000F731127E02E8C8D8E110CC00FB607FC19
:1003D000FACFE889F989808185FFF5CFCE010E94A7
:1003E0009201F1CFEB8DEC0FFD2FF11DE35AFF4F82
:1003F000F0829FB7F8940B8FEA89FB898081806235
:10040000CFCF682F88E591E00C94B401CF93DF93B0
:10041000EC01888D8823B9F0AA89BB89E889F9891C
:100420008C9185FD03C0808186FD0DC00FB607FC51
:10043000F7CF8C9185FFF2CF808185FFEDCFCE0184
:100440000E949201E9CFDF91CF91089561E082E0AF
:100450000C94B50060E082E00C94B500CF93DF937C
:10046000D82FC8E06D2F617085E00E94B500D69549
:1004700061E088E00E94B50060E088E00E94B5007D
:10048000C15081F7DF91CF910895CF93C82F60E0DD
:1004900082E00E94B5008C2F0E942E0261E082E073
:1004A000CF910C94B5000C942E02CF93DF93D82FEC
:1004B000E62FF0E0EE5DFE4FC08181818111C260C8
:1004C00082818111C46083818111C860848181111E
:1004D000C06185818111C06286818111C06487817C
:1004E0008111C06884E40E9445020E942A0287E0CC
:1004F0008D1B880F80540E9453028C2F0E94530240
:10050000DF91CF910C9426029F92AF92BF92CF922F
:10051000DF92EF92FF920F931F93CF93DF93D0E080
:10052000C0E0B12C03EB10E09FE9E92E90E0F92E3A
:100530002BE8C22E20E0D22E61E088E00E94B500B8
:10054000F8018491F701A490F6019490992061F14B
:1005500081110E948C00E92DF0E0EE0FFF1FE4589E
:10056000FF4FA591B4918C91A82231E009F430E0BD
:10057000832F0C2E01C0880F0A94EAF7B82A60E096
:1005800088E00E94B5002196C830D105A9F68B2DD0
:10059000DF91CF911F910F91FF90EF90DF90CF905F
:1005A000BF90AF909F90089580E0E3CFFC01019051
:1005B0000020E9F73197AF01481B590BBC0188E5D2
:1005C00091E00C9414018F929F92AF92BF92CF92C0
:1005D000DF92EF92FF920F931F93CF93DF93CDB7EC
:1005E000DEB7A1970FB6F894DEBF0FBECDBF6B018B
:1005F0007C01F7FE41C06DE288E591E00E94B40104
:100600008C0122273327A9012C193D094E095F09C6
:1006100019A2CE0181967C019AE0892E912CA12C01
:10062000B12CCA01B901A50194010E942206605DA6
:10063000F70162937F01211531054105510589F7C5
:1006400090E080E0309719F0CF010E94D602800F31
:10065000911FA1960FB6F894DEBF0FBECDBFDF91FC
:10066000CF911F910F91FF90EF90DF90CF90BF90AF
:10067000AF909F908F900895AC019B0119A28E01BD
:100680000F5D1F4F8AE0C82ED12CE12CF12CCA013E
:10069000B901A70196010E942206605DF8016293EC
:1006A0008F01211531054105510589F790E080E062
:1006B000309779F2CF010E94D602CBCF1F920F92D2
:1006C0000FB60F9211242F933F938F939F93AF9365
:1006D000BF938091540190915501A0915601B09122
:1006E00057013091530123E0230F2D3758F5019620
:1006F000A11DB11D20935301809354019093550186
:10070000A0935601B093570180914F0190915001F1
:10071000A0915101B09152010196A11DB11D80938C
:100720004F0190935001A0935101B0935201BF919A
:10073000AF919F918F913F912F910F900FBE0F908E
:100740001F90189526E8230F0296A11DB11DD2CF48
:100750001F920F920FB60F9211242F933F934F9336
:100760005F936F937F938F939F93AF93BF93EF9319
:10077000FF9388E591E00E949201FF91EF91BF9174
:10078000AF919F918F917F916F915F914F913F9129
:100790002F910F900FBE0F901F9018951F920F92E0
:1007A0000FB60F9211242F938F939F93EF93FF9384
:1007B000E0916801F09169018081E0916E01F09112
:1007C0006F0182FD1BC09081809171018F5F8F73DB
:1007D00020917201821741F0E0917101F0E0E85A36
:1007E000FE4F958F80937101FF91EF919F918F91B3
:1007F0002F910F900FBE0F901F9018958081F4CF0E
:10080000789484B5826084BD84B5816084BD85B5EB
:10081000826085BD85B5816085BD80916E008160F7
:1008200080936E001092810080918100826080939D
:10083000810080918100816080938100809180009F
:100840008160809380008091B10084608093B100CA
:100850008091B00081608093B00080917A008460C4
:1008600080937A0080917A00826080937A008091F0
:100870007A00816080937A0080917A00806880930A
:100880007A001092C100E0916801F091690182E064
:100890008083E0916401F09165011082E09166012E
:1008A000F09167018FEC808310927001E0916C01F0
:1008B000F0916D0186E08083E0916A01F0916B0117
:1008C000808180618083E0916A01F0916B01808179
:1008D00088608083E0916A01F0916B01808180687B
:1008E0008083E0916A01F0916B0180818F7D80832C
:1008F00061E082E00E94E30061E088E00E94E300A2
:1009000061E085E00E94E30061E082E00E94B500C2
:1009100061E088E00E94B50061E085E00E94B500DA
:1009200080E40E9445020E942A0280EC0E94530249
:10093000C0E180E00E945302C150D9F70E94260214
:100940008FE80E9445028CE80E94450298E0B92E8B
:1009500020E0E22E20E0F22E0E942A0282E40E9491
:10096000530260E085E00E94E300CAE1D1E08EE03E
:10097000882E912C0E948402982F9170792E829556
:100980008170A82E8B81A81699F0AB8282E191E04C
:100990000E94D602B401685071096A29072E000C22
:1009A000880B990B0E94E30284E191E00E94D60239
:1009B0008F81781689F07F8282E191E00E94D602D1
:1009C000B4016729072E000C880B990B0E94E302E3
:1009D00084E191E00E94D602219782E0881A910872
:1009E00096E08916910431F661E085E00E94E3000B
:1009F0000E94260288E591E00E94720118161906ED
:100A000054F488E591E00E9450018F36910569F514
:100A100081E080934E0180914E01882309F4D9C072
:100A2000C0904C01D0904D01C6010197089708F085
:100A3000C7C0F601EF5DFE4FA08084E40E9445022E
:100A40000E942A028B2D8C19880F8F530E9453020B
:100A50008A2D0E9453020E9426028AE1C816D10400
:100A600009F0A1C062E181E0B2C08A30910539F499
:100A700010924E0110924D0110924C01CCCF20915A
:100A80004E012223B1F020914C0130914D012A32C8
:100A900031057CF4F901EE5DFE4F41E0C09709F4A9
:100AA00040E040832F5F3F4F30934D0120934C0136
:100AB000B2CF8337910509F054C00E942A0282E424
:100AC0000E94530260E085E00E94E300D12CC12C1B
:100AD000812C0E94840280FB442440F8512C920116
:100AE0000C2C01C0220F0A94EAF780710C2C01C073
:100AF000880F0A94EAF7822B882A8FEFC81AD80A3F
:100B000094E0C916D10429F787E191E00E94D6024A
:100B1000D12CC12C912CC4010C2C01C0880F0A943B
:100B2000EAF787FB002700F910E0B801110F880BE6
:100B3000990B0E94E3028FEFC81AD80A98E0C916F1
:100B4000D10449F786E191E00E94D60284E191E068
:100B50000E94D60261E085E00E94E3000E94260226
:100B60005ACF8637910509F056CF66E788E591E0C0
:100B70000E94B40181E090E00E94010281E090E0D7
:100B80000E94010290E080E00E94010290E080E07B
:100B90000E94010286E191E00E94D60284E191E088
:100BA0000E94D60238CF6AE182E092E2C916D104EF
:100BB00071F08AE2C816D10461F462E283E007C0F2
:100BC00092E1C916D10409F048CF6AE080E00E94A2
:100BD0005502E114F10409F4BFCE0E947E0188237E
:100BE00009F4BACE0E940000B7CEE8E5F1E0138226
:100BF000128288EE93E0A0E0B0E084839583A68320
:100C0000B78384E091E09183808385EC90E09587C1
:100C1000848784EC90E09787868780EC90E0918BC6
:100C2000808B81EC90E0938B828B82EC90E0958BB3
:100C3000848B86EC90E0978B868B118E128E138EB0
:100C4000148E0895A1E21A2EAA1BBB1BFD010DC034
:100C5000AA1FBB1FEE1FFF1FA217B307E407F5076C
:100C600020F0A21BB30BE40BF50B661F771F881F48
:100C7000991F1A9469F760957095809590959B01DE
:100C8000AC01BD01CF010895EE0FFF1F0590F49157
:080C9000E02D0994F894FFCF58
:100C980000000000B4011401410106027201500174
:0A0CA800640169000D0A00730000EA
:00000001FF
